:020000005E2878
:0800080090000308910083122F
:10001000930803199203930313081204031D4C2839
:10002000AD0AAE0A2915940B482825089400A91595
:100030000130AE00AA1C262803302502031D242807
:10004000A5030130AD004828A50A48282A1D3528F7
:1000500003302502031D3128A5032B100130AD000C
:1000600048282B18A50A2B144828AA1D4628023018
:100070002502031D3E28A50A2B1048282B1C4228C8
:10008000A50348282B140130AD0048280130AD00ED
:100090001508920016089300970B57281808970028
:1000A000A20AA91F5728A80B5728A91329160B1114
:1000B000640011088300900E100E09008101830175
:1000C000053084008001840A50300402031D622838
:1000D00084018501831685018312860183168113AD
:1000E0008601831205168511B322A001A2012730D3
:1000F000980097007830A4000330A50001309400E8
:100100000A30A6000430A7006D21A901AA01291414
:10011000A914AA17C3222030AB222030AB222030F2
:10012000AB222030AB224530AB224C30AB224530E5
:10013000AB224B30AB225430AB224F30AB2252308B
:10014000AB222030AB22FA30C722FA30C722FA3075
:10015000C722FA30C72205228316811281150B119E
:100160008B168B178312A91BBB28291DBB28AD2119
:100170009321A9112911291FBF280522291323081A
:100180002202031CD328A20129212A1BD328A0184C
:10019000D9202019E520A01AED20A01BF420201B57
:1001A000FB20201ADD2A291ED8286D2129172912A3
:1001B000B328A40AF0302402031CE028F030A40085
:1001C00029176430A800A9170800A40328302402C6
:1001D0000318E0282830A400E028A91CF128A91061
:1001E000F228A914291708002918F8282914F92831
:1001F000291029170800AA1C0029AA102A15182955
:100200002A1D05292A11AA151829AA1D0C29023010
:10021000A5002A14AA1118292A1C10292A10182905
:10022000A50A08302502031D1829AA140330A500C9
:10023000013094002917080085108316F6308600D7
:100240008312051206080516FF3A831686018312EB
:1002500008002A1B33291C212006A1002A17A2010D
:100260000230A30008001C212006A1052108A006D9
:10027000F630A005A105AA1F452920082105031D68
:10028000582920080639031D49292008031D58292B
:1002900055292308053C03195A290F30A302031CD2
:1002A00055290530230203185A290530A3005A297D
:1002B0003230A3002A130800B801B901BA00643033
:1002C0003A02031C6629BA00B80A5F290A303A02CA
:1002D000031C0800BA00B90A5F298B130330B4006D
:1002E0009330B5008730B600B3011830B700031063
:1002F000B60DB50DB40DB30D0318822924083302D1
:10030000031C85292408B3023614B70B7729350856
:1003100095003608960015089200160893000130E3
:1003200094008B170800A91997292A1CA6292918B7
:100330000515A91CA0290330BC006B30F321A229AC
:100340003230C7223230C7220511AC29A91CAC2992
:100350000430BC007230F32108002C08C038AF22F2
:100360002030AB222D0BB629AC01D529AA1DBB2903
:100370000230AC07D529AA1CC0290430AC07D52906
:100380002A1DC5290530BF00C82902302502BF003B
:100390002D1CD02901308A003F08E521AC07D52962
:1003A00001308A003F08EC21AC070F302C02031CFF
:1003B000DB290F30AC002C08C038AF222A1CE22900
:1003C000FF30AB2A2E083038AB2A820700340834BD
:1003D000053404340334023482070F3407340534FF
:1003E000043403340334BB00BB030310BB0CFF30E5
:1003F0008600851585113B08D0228601851585115B
:100400003B08D022BC0BF7290800C3222A1E1F2A52
:100410005430AB184630AB22C030AF2202308A00D5
:10042000260826076322AB22260A26076322FF3905
:1004300003191B2AAB2227083038AB224F2A240885
:100440005C2138083038AB2239083038AB223A0802
:100450003038AB228430AF22AA1C302A3530372AFC
:100460002A1D342A3730372AAA1D3D2A3830AB22BC
:100470002F30AB223430AB22482A2030AB222A1C4A
:10048000432A3130472A25085C213A083038AB220C
:100490008D30AF22291C4E2A57224F2A5D228830E8
:1004A000AF22A91C552A5722562A5D2208004F3038
:1004B000AB226E30AB222030AB2A4F30AB226630FD
:1004C000AB226630AB2A8207003400344334003458
:1004D0004334233444340034443423344534003426
:1004E000463400344634233447340034473423340C
:1004F0004134003441342334423400349C008316A8
:10050000F030860483128611051400008514000063
:1005100006089A0085109A1F912A851400008510FC
:10052000862A85140000851083160F3086058312F5
:100530001C0808009C009A009A0EA0221C089A0031
:1005400085140F309A0586059A0E1A088604000055
:1005500085100530D02A7E22051086159A2A7E2223
:10056000051086119A2A0F30C7222030AF2205309D
:10057000C7222030AF220A30D0220630AF220C3002
:10058000AF220130AF2A0130AF220230C72A9E00CD
:10059000F9309F0000009F0BCA2A9E0BC82A080052
:1005A0009E009E0BD42ADB2A02309F009F0BD62A86
:1005B0009E0BD42ADB2A000008008B132A160A306F
:1005C000A6000430A70005220516A0012016B101DF
:1005D000B20161232F08B1070318B20A3008B2072D
:1005E00003308A003208321BFF3A3F39AC23B21B7A
:1005F000FF3A8600A918851585118316F630860006
:100600008312051206080516831686018312FF3A27
:100610002006F6390319EA2A1C21A0001430C7224B
:100620001C21A0050319EA2AA018422B2019532BDC
:10063000A01A3C2BA01B2A2B201B342B201A212B69
:10064000EA2AAB1C282BAB102A128B172917B328C8
:10065000AB14312BA70A08302702031C312B0730BB
:10066000A70061230522EA2AA70302302702031804
:10067000312B0230A700312BA91C402BA910312BA4
:10068000A914312BA60A0D302602031C312B013090
:10069000A600A70A08302702031C312B0730A70049
:1006A0000C30A600312BA60B312B0C30A600A70373
:1006B000023027020318312B0230A7000130A600B8
:1006C000312B03308A002603AB180C3E7A23AF008F
:1006D00003308A002603AB180C3E9323B000270892
:1006E000073C0319792BBF000310B00CAF0CBF0BF4
:1006F000742B080082076F34B5340F347D34013415
:100700009C344F341D3405340B34303475345C3430
:1007100081340834513408347B346A340A34C134A7
:100720000B34F9348D3482071534163418341934E7
:100730001B341C341E342034223424342634283410
:1007400015341634183419341B341C341E34203438
:100750002134243425342834820780348334863489
:1007600089348C3490349334963499349C349F3447
:10077000A234A534A834AB34AE34B134B334B63477
:10078000B934BC34BF34C134C434C734C934CC34B4
:10079000CE34D134D334D534D834DA34DC34DE3406
:1007A000E034E234E434E634E834EA34EB34ED3473
:1007B000EF34F034F134F334F434F534F634F834FF
:1007C000F934FA34FA34FB34FC34FD34FD34FE34AD
:0C07D000FE34FE34FF34FF34FF34FF34ED
:02400E00F13F80
:00000001FF
